:020000040800F2
:1000000090760020B1010008B10E00082D0D000807
:100010009D0E0008A70200086D17000800000000F0
:10002000000000000000000000000000D1110008E6
:10003000950A000800000000410F0008E9120008BE
:10004000CB010008CB010008CB010008CB01000860
:10005000CB010008CB010008CB010008CB01000850
:10006000CB010008CB010008CB010008CB01000840
:10007000CB010008CB010008CB010008CB01000830
:10008000CB010008CB010008CB010008CB01000820
:10009000CB010008CB010008CB010008CB01000810
:1000A000CB010008CB010008CB010008CB01000800
:1000B000CB01000855130008CB010008CB01000854
:1000C000CB010008CB010008CB010008CB010008E0
:1000D000CB010008CB010008CB010008CB010008D0
:1000E000CB010008CB010008CB010008CB010008C0
:1000F000CB010008CB010008CB010008CB010008B0
:10010000CB010008CB010008CB010008CB0100089F
:10011000CB010008CB010008CB010008CB0100088F
:10012000CB010008CB010008CB010008CB0100087F
:10013000CB010008CB010008CB010008CB0100086F
:10014000CB010008CB010008CB010008CB0100085F
:10015000CB010008CB010008CB010008FD1300080B
:10016000CB010008CB010008CB010008CB0100083F
:10017000CB010008CB010008CB010008CB0100082F
:10018000CB010008CB010008DFF810D000F04EF8DA
:10019000004800475D1A0008AFF300809076002009
:1001A00030BF72B6704762B6704780F308887047F8
:1001B0000648804706480047FEE7FEE7FEE7FEE701
:1001C000FEE7FEE7FEE7FEE7FEE7FEE7ED120008CA
:1001D0008901000840EA01039B0703D009E008C930
:1001E000121F08C0042AFAD203E011F8013B00F8FC
:1001F000013B521EF9D27047D2B201E000F8012B48
:10020000491EFBD270470022F6E710B513460A4696
:1002100004461946FFF7F0FF204610BD421C10F8B7
:10022000011B0029FBD1801A70470000064C074DC6
:1002300006E0E06840F0010394E8070098471034B6
:10024000AC42F6D3FFF7A4FFB41B0008D41B000890
:1002500070B58C1810F8015B15F0070301D110F888
:10026000013B2A1106D110F8012B03E010F8016BB5
:1002700001F8016B5B1EF9D12B0705D40023521E38
:100280000DD401F8013BFAE710F8013BCB1A921CA0
:1002900003E013F8015B01F8015B521EF9D5A1429E
:1002A000D8D3002070BD00BFFEE700002DE9F0416B
:1002B00006460F4690461C46012511200449087049
:1002C00022462946012001F06BF9BDE8F0810000CB
:1002D000C44500202DE9F05F81468A4693461E46BC
:1002E000812739463448FFF78EFF00F01BFD044696
:1002F00020783149087060784870A07888700020B4
:1003000005E0211D0A5CC11C2B4B5A54401C0E28D1
:10031000F7DB04F11200FFF781FF0546102D01DD28
:10032000102000E028460546002007E004F11201F5
:100330000A5C00F11101204B5A54401CA842F5DB25
:1003400004F12200FFF76AFF0546202D01DD202081
:1003500000E028460546002007E004F122010A5C7F
:1003600000F12101144B5A54401CA842F5DB04F162
:100370004200FFF753FF0546402D01DD402000E01D
:1003800028460546002007E004F142010A5C00F11E
:100390004101094B5A54401CA842F5DB074B3A4631
:1003A0000549032000F0C5FA80463246394602204E
:1003B00001F0F6F8BDE8F09FC4450020C44D0020D0
:1003C0002DE9F05F81468A4693461E4681273946CD
:1003D0003448FFF718FF00F0A5FC044620783149A7
:1003E000087060784870A0788870002005E0211DB2
:1003F0000A5CC11C2B4B5A54401C0E28F7DB04F13D
:100400001200FFF70BFF0546102D01DD102000E064
:1004100028460546002007E004F112010A5C00F1BD
:100420001101204B5A54401CA842F5DB04F1220074
:10043000FFF7F4FE0546202D01DD202000E02846D0
:100440000546002007E004F122010A5C00F12101C9
:10045000144B5A54401CA842F5DB04F14200FFF74C
:10046000DDFE0546402D01DD402000E02846054622
:10047000002007E004F142010A5C00F14101094B50
:100480005A54401CA842F5DB074B3A460549032065
:1004900000F04FFA804632463946032001F080F8DA
:1004A000BDE8F09FC4450020C44D00202DE9F04177
:1004B000AAB006460F4690461C460E2501A801F03C
:1004C000F1F92A460DF18E010548FFF783FE224619
:1004D0002946042001F064F82AB0BDE8F08100004C
:1004E000C44500202DE9F04704460E4617461D4638
:1004F00000201D4908704FF001094FF001081DB19F
:100500004FEA48604FEA10683FB13146204600F09C
:1005100073FC10B94FF000091BE0022E02DA4FF015
:10052000000916E020781149087000201049087071
:1005300010490870104908600C480078772804D0EA
:10054000607810B90D4801F013FA012006490870CF
:1005500000BF0B4880F800902A464146052001F074
:100560001FF8BDE8F0870000B4010020B5010020AD
:10057000B6010020B7010020B801002000000C08DF
:10058000C44500202DE9F04105460C461646984624
:1005900027465EB12146284600F02EFC08B9BDE88A
:1005A000F081204604EBD071C1F34F07142F07DA16
:1005B000002003E0295C034A1154401CB842F9DBD7
:1005C00000BFECE7A00100202DE9F04106460F46F0
:1005D00090461C4614252A4605490648FFF7FAFDB1
:1005E00022462946072000F0DBFFBDE8F08100002D
:1005F000A0010020C44500202DE9FF4F83B0044630
:1006000089462C48007830B90121062000F034FAE0
:1006100007B0BDE8F08F4FF0000AA9F108052E469B
:100620003546615D701C205C01EB0021B01C205C34
:1006300001EB0041F01C205C01EB006B2F1DE15D24
:10064000781C205C01EB0021B81C205C01EB004110
:10065000F81C205C01EB006002903946204600F057
:100660008BFB80460298404502D04FF0FF0A15E010
:1006700011480078772805D12A462146584601F0CE
:100680009FF904E02A462146584601F0A7F90B4895
:1006900000682844094908604FF0000A01200190D1
:1006A000074880F800A00820069A019900F078FF1A
:1006B00000BFADE7B4010020B5010020B801002063
:1006C000C44500202DE9F05F044699462148007892
:1006D00028B90121062000F0CFF9BDE8F09F0025E0
:1006E000615D681C205C01EB0021A81C205C01EB13
:1006F0000041E81C205C01EB00672E1DA15D701C11
:10070000205C01EB0021B01C205C01EB0041F01CDF
:10071000205C01EB006AA8460F480068B84209D186
:1007200039460E4800F03EFB8046C24502D101200A
:100730000B4908704FF0080B0A4807490968016027
:10074000C0F804804A4659460B2000F029FF00BF3C
:10075000C3E70000B4010020B801002000000C082D
:10076000B6010020C44500202DE9F84F81468A4695
:1007700093461E4600251548007800B901251DB98D
:100780001348007800B90125ADB912480068C01CB3
:100790004FEA900800240BE00F4951F82400009024
:1007A0000E4901EB84000122694600F0C3FC641C81
:1007B0004445F1D300BF0127094805703246394648
:1007C0000C2000F0EDFEBDE8F88F0000B401002021
:1007D000B6010020B801002000000C08000002084B
:1007E000C44500202DE9FC478046894692461C46B8
:1007F00018480068C01C8708002500201DE0164A24
:1008000052F820100191154A52F820100091DDE9AC
:10081000002191420DD0810006E00E4A12689142FB
:1008200001D2012504E003E0421CB1EB820FF4D3B6
:1008300000BF012D00D102E0401CB842DFD300BF51
:10084000012607480570224631460D2000F0A8FE1B
:10085000BDE8FC87B80100200000020800000C0879
:10086000C4450020F0B5A9B004460D4616461F4603
:1008700077201049087000200F490870684601F081
:1008800011F8FF208DF80100684601F015F80B48BB
:10089000406800F07F40B0F1006F05D101F07EF8B4
:1008A000064801F065F803E0034800780249087043
:1008B00029B0F0BDB5010020B401002000000208FD
:1008C0002DE9F043A9B005460C4616469946012786
:1008D00004F0FF0856B1204604EBD071C1F347087D
:1008E0002146284600F088FA00B90027B8F10E0F1B
:1008F00000DA002767B1684600F0D4FF0E222946CF
:100900000DF18A00FFF766FC684600F0D5FF03E0B2
:100910000121022000F0B0F829B0BDE8F0832DE9F4
:10092000F04104460D4616461F4600F039FDBDE86D
:10093000F0812DE9F04106460F4615461C4655202C
:100940002070AA206070BB20A070E6702571280A74
:100950006071002D04DD2A463946A01DFFF73AFCE0
:100960000D21A81D21540A21E81D2154401CBDE879
:10097000F08100002DE9F0413A483B49097830F810
:1009800011604FF6FF70864200D15FE04FF6FF70B6
:100990003449354A127821F8120000200CE033491E
:1009A000895D334A1154711C44F2080291FBF2F341
:1009B00002FB13118EB2401CB0F5026FEFDB2C4826
:1009C0000078552807D12A484078AA2803D128481A
:1009D0008078BB2800D039E0254DA888801D2946A5
:1009E000085C0D2804D1A888C01D085C0A2800D026
:1009F0002CE01C481C49097830F811601C4F002479
:100A000020E004EB44001B4911F82000F9788842EB
:100A100016D104EB4400DFF85C8008EB8000437AD9
:100A200004EB440008EB8000027AB98804EB440030
:100A300008EB8000D0F804C00D48801DE04703E0BB
:100A4000601CC4B21E2CDCDB00BF00BF064800786F
:100A5000401C142190FBF1F201FB120002490870C6
:100A6000BDE8F0814456002009000020BC050020AC
:100A70006C5E00203000002070B504460D46012653
:100A8000034804702A463146B02000F089FD70BD4D
:100A9000C44500207047000001490860704700000D
:100AA0000C3C024030B10749096841F48061054AB5
:100AB000116005E00349096821F48061014A116071
:100AC00070470000003C024070B504460A4600260C
:100AD000092502B909E0012A01D1160205E0022A1E
:100AE00001D1160201E04FF4407600F09FF8054670
:100AF000092D28D11548006820F44070134908607A
:100B000008460068304308600846006820F0F80096
:100B100008600846006844F0020108430B49086079
:100B20000846006840F48030086000F07FF8054611
:100B30000648006820F00200044908600846006882
:100B400020F0F8000860284670BD0000103C02400C
:100B500009201349096801F48031B1F5803F01D1C2
:100B600001201CE00E49096801F0100109B10620BE
:100B700015E00B49096801F4807109B102200EE00B
:100B80000749096801F0EF0109B1072007E00449AE
:100B9000096801F0020109B1082000E0092070474E
:100BA0000C3C02400348006840F0004001490860E6
:100BB00070470000103C024030B502460C46092543
:100BC00000F034F80546092D19D10E48006820F4CC
:100BD00040700C4908600846006840F400700860E6
:100BE0000846006840F001000860146000F01EF83C
:100BF00005460448006820F00100024908602846C4
:100C000030BD0000103C02400548006800F0004084
:100C100028B1044802490C3908600348086070474D
:100C2000103C024023016745AB89EFCD08B5092090
:100C30000090FFF78DFF009002E0FFF789FF009022
:100C40009DF800000128F8D09DF8000008BDF0B51F
:100C50000A4600210023002400BF3DE0012505FADB
:100C600001F3156805EA03049C4234D105684F007E
:100C70000326BE40B543056015794E00B5400668B1
:100C8000354305601579012D02D01579022D16D155
:100C900085684F000326BE40B543856055794E00F8
:100CA000B540866835438560456801268E40B5436A
:100CB0004560456896798E40B6B235434560C56853
:100CC0004F000326BE40B543C560D5794E00B54000
:100CD000C6683543C560491C1029BFD3F0BDF0B5C7
:100CE000002300244D07ED0E02FA05F3CE1000F1AB
:100CF000200555F826504E07F70E0F26BE40B54387
:100D0000CF1000F1200646F82750CE1000F1200544
:100D100055F8265045EA0304CE1000F1200545F8A9
:100D20002640F0BD00487047301B000802480349C8
:100D3000086000BFFEE700000400FA050CED00E0CB
:100D4000002111E00846082208E000F001031BB171
:100D5000074B83EA500000E04008521E002AF4DCF2
:100D6000044B43F82100491CFF29EBDD70470000CC
:100D70002083B8EDBC01002030B502460B464FF091
:100D8000FF31002008E0CCB2155C6C40044D55F8F2
:100D9000244084EA1121401C9842F4D3C84330BD5A
:100DA000BC010020F8B504464FF0FF32C81C86088D
:100DB0000025002019E054F820300093002310E0B3
:100DC0008D420CD2D7B21DF803C087EA0C07DFF8BA
:100DD00024C05CF8277087EA12226D1C00E002E054
:100DE0005B1C042BECD300BF401CB042E3D3D043C8
:100DF000F8BD0000BC01002030B5034609B9012050
:100E000030BD084601EBD0725210A1EB42020AB18C
:100E10000020F5E7084601EBD072C2F34F04002230
:100E200009E0985CC043C0B215195D5DA84201D0CD
:100E30000020E5E7521CA242F3DB0120E0E710B5F9
:100E40000246002004E0135CDB4344181355401CA9
:100E50008842F8DB10BD000010B54FF4A06000F030
:100E600065F8A82000F094FC4FF4E13000F004FE97
:100E700001200849087000F069FD012809D10648E1
:100E8000406800F07F40B0F1006F02D1024800F0EE
:100E90006FFD10BD04000020000002080248034955
:100EA000086000BFFEE700000400FA050CED00E05A
:100EB0007047000070B5002100230F22C4781CB3D6
:100EC000174C246804F4E064C4F5E064C4F307211B
:100ED000C1F10404E3B20A4144789C40E1B2847851
:100EE000144021430C07210E0E4C057861550478FF
:100EF00004F01F050124AC4005786D11AD0005F12B
:100F0000E025C5F8004109E0047804F01F0501243C
:100F1000AC40054D0678761145F8264070BD0000BE
:100F20000CED00E000E400E080E100E00249014354
:100F3000024A1160704700000000FA050CED00E065
:100F40007047000029B1064A12680243044B1A6038
:100F500004E0034A12688243014B1A6070470000A4
:100F60003038024029B1064A12680243044B1A6025
:100F700004E0034A12688243014B1A607047000084
:100F800044380240F0B5002100220024022500264A
:100F90000223324F3F6807F00C0121B1042905D02C
:100FA000082937D105E02E4F076036E02D4F076046
:100FB00033E02A4F3F1F3F68C7F38056274F3F1F3C
:100FC0003F6807F03F036EB1264FB7FBF3F7DFF83A
:100FD0008CC0ACF1040CDCF800C0CCF3881C07FB1F
:100FE0000CF40CE01E4FB7FBF3F7DFF870C0ACF168
:100FF000040CDCF800C0CCF3881C07FB0CF4174F82
:101000003F1F3F68C7F301477F1C7D00B4FBF5F726
:10101000076002E0124F076000BF00BF0F4F3F683C
:1010200007F0F0010909104F7A5C0768D740476064
:101030000A4F3F6807F4E051890A0B4F7A5C476812
:10104000D7408760054F3F6807F46041490B064F62
:101050007A5C4768D740C760F0BD0000083802409E
:101060000024F40000127A002000002001461C48F1
:10107000814201D2002070471A48814201D20820E3
:10108000F9E71948814201D21020F4E7174881425C
:1010900001D21820EFE71648814201D22020EAE76A
:1010A0001448814201D22820E5E71348814201D249
:1010B0003020E0E71148814201D23820DBE71048B8
:1010C000814201D24020D6E70E48814201D2482019
:1010D000D1E70D48814201D25020CCE75820CAE721
:1010E000004000080080000800C00008000001085F
:1010F00000000208000004080000060800000808BC
:1011000000000A0800000C0800000E0830B5034675
:101110000C461546002206E0184600F007F844F891
:1011200022001B1D521CAA42F6D330BD014608689E
:10113000704700002DE9F04704460E4617464FF071
:1011400009080025A946B4F1006F02D304F003009A
:1011500008B1BDE8F087FFF757FD0020FFF7A2FCBC
:10116000254604EB87091948854218D214E0284621
:10117000FFF7DCFF401C70B1F120FFF78DFC284623
:10118000FFF774FF82460221FFF79EFC8046B8F10C
:10119000090F01D002E02D1D4D45E8D300BFB8F185
:1011A000090F0CD108E020463168FFF705FD09283A
:1011B00000D003E0241D361D4C45F4D300BF0120B0
:1011C000FFF770FCFFF7EEFC00BFC2E70000FF1F57
:1011D000704700000CB50020019000903448006872
:1011E00040F480303249086000BF3148006800F4A4
:1011F000003000900198401C0190009818B90198A7
:10120000B0F5A04FF1D12A48006800F4003010B1C9
:101210000120009001E0002000900098012846D1B4
:1012200023484030006840F0805021494031086038
:101230002048006840F440401E4908601C480830BF
:1012400000681B49083108600846006840F4004007
:1012500008600846006840F4A05008601648091F5E
:101260000860081F006840F08070091F086000BF18
:101270000F48006800F000700028F9D040F20570B7
:101280000E4908600A480830006820F00300084949
:10129000083108600846006840F00200086000BF9E
:1012A00003480830006800F00C000828F8D10CBD95
:1012B000003802400070004008544007003C0240E3
:1012C000042808D14FF0E021096941F004014FF0F2
:1012D000E022116107E04FF0E021096921F00401EB
:1012E0004FF0E022116170477047000010B51548BB
:1012F000006840F47000134908601348006840F02B
:1013000001001149086000200F49083108600E48AB
:1013100000680E4908400C4908600D48091D086026
:10132000081F006820F48020091F0860002006497B
:101330000C310860FFF74EFF4FF000600149803923
:10134000086010BD88ED00E000380240FFFFF6FEA7
:101350001030002410B50121054800F010F80128D4
:1013600001D1044908700121014800F005F810BDC1
:101370000004004018000020CA430282704730B5C4
:101380000246002000230024158A05EA01039589FE
:1013900005EA010413B10CB1012000E0002030BDCA
:1013A000002005E04FF6FF710B4A22F81010401C98
:1013B0001428F7DB00200949087009490870094919
:1013C00008700949086009490870094908800949F5
:1013D0000880094908807047445600200A00002010
:1013E00008000020090000200C0000201000002050
:1013F0001200002014000020160000205E49098819
:1014000001F0200121B15C49091D0988C8B200E042
:1014100070475A4909780A297BD2DFE801F005179D
:10142000232F353B4E52616D55280ED10121544A70
:101430001170544A11800021534A118001214F4AF2
:10144000117052490988524A118063E0AA2803D1D9
:1014500002214A4A117004E00021494A1170474AAA
:10146000117057E0BB2803D10321444A117004E0F6
:101470000021434A1170414A11704BE004213F4A58
:1014800011704149088045E005213C4A11703E49F0
:1014900008803FE00621394A11703B49098841EA3A
:1014A0000021394A11800021364A118036490988C5
:1014B00011B90821314A11702CE007212F4A11700F
:1014C00000BF30490988491C2E4A118011460988FD
:1014D0002D4A1288914202DB0821284A117019E036
:1014E0000D2805D00021264A1170244A117002E00F
:1014F0000921224A11700DE00A2806D00021204A55
:1015000011701E4A117003E003E00A211B4A11709A
:1015100000E000BF00BF1A49097881B11B490A6881
:101520000968491C194B19601A49885419460968F9
:1015300044F20802914202D300211A4611600F4979
:1015400009780A2915D112490988134A134B1B78C7
:1015500022F8131011490978491C142291FBF2F367
:1015600002FB13110D4A11700021054A1170034A44
:10157000117000BF4CE70000001401400A00002079
:101580001000002016000020140000200C00002095
:1015900012000020BC050020445600200800002056
:1015A0002DE9F04781460C461646274626B1A1B2E2
:1015B0001048FFF744FC7F000F4B3A460D49484660
:1015C000FFF7B7F9804640210C4800F019F80025D4
:1015D0000CE00948415D094800F0C4F800BF402113
:1015E000064800F022F80128F9D16D1C4545F0DBD2
:1015F000BDE8F087C4450020C44D00200014014020
:1016000001F40072B2F5007F00D100BFCA4302802E
:10161000704721B1828942F40052828104E08289BC
:101620004DF6FF731A408281704702460020B1F5E3
:10163000007F00D100BF13880B400BB1012000E0F8
:1016400000207047F0B50346002400260025002046
:1016500040F66A17B94200D100BF1846C1F34214E0
:1016600001F01F06012707FA06F5012C01D10C3005
:1016700004E0022C01D1103000E014301AB10768E8
:101680002F43076002E00768AF430760F0BD00002A
:101690002DE9FF4705460E460024A14600BFA0469F
:1016A000B08900B100BF2C8A24F44054F088044370
:1016B0002C82AC8941F20C608443B08831890843A4
:1016C000718908430443AC81AC8A24F44074B08926
:1016D0000443AC826846FFF755FC2048854202D09F
:1016E0001F48854202D1DDF80C9001E0DDF808903A
:1016F000A88900F4004040B109EBC90000EB0910D3
:1017000031684900B0FBF1F707E009EBC90000EBD5
:10171000091031688900B0FBF1F76420B7FBF0F0E5
:1017200004012009642101FB1078A88900F400401D
:1017300040B1322000EBC800B0FBF1F000F0070030
:10174000044308E0322000EB08106421B0FBF1F004
:1017500000F00F0004432C81BDE8FF87001001401A
:1017600000140140C1F308028280704700BFFEE709
:1017700002E008C8121F08C1002AFAD1704770475A
:10178000002001E001C1121F002AFBD170470000B8
:1017900010B504466FF00400FFF792FDE11704EB6B
:1017A0005171C1F3C701074A11701046007800EB70
:1017B0004001C1EBC0104FF6FF7101EAC0000249C1
:1017C000088010BD000000200200002070B5044613
:1017D0004FF4077094FBF0F0C6B24FF4077094FB1F
:1017E000F0F100FB114085B204B970BD05E04FF483
:1017F000077000F031F8701EC6B2002EF7D115B197
:10180000284600F029F800BFEFE700000146114A22
:1018100012784A434FF0E0235A6100229A611A4637
:10182000126942F001021A6100BF4FF0E022106914
:1018300000F001021AB100F48032002AF5D04FF016
:10184000E022126922F001024FF0E0231A61002227
:101850009A617047000000200146114A12884A43ED
:101860004FF0E0235A6100229A611A46126942F051
:1018700001021A6100BF4FF0E022106900F001027E
:101880001AB100F48032002AF5D04FF0E02212693C
:1018900022F001024FF0E0231A6100229A617047A2
:1018A0000200002010B50446282221460148FFF717
:1018B0002DFC10BD0000010810B504462822214669
:1018C0000148FFF737FC10BD0000010810B5AAB0B1
:1018D00001A8FFF7E7FF9DF80400FF2803D09DF85B
:1018E0000500FF282FD1FFF71DFA044620788DF858
:1018F000040060788DF80500A0788DF80600E07887
:101900008DF807000E22211D02A8FEF763FC20229D
:1019100004F122010DF12600FEF75CFC0E2204F119
:1019200012010DF11600FEF755FC402204F14201B0
:101930000DF14600FEF74EFC01A8FFF7BDFF0A209F
:10194000FFF744FF00BF2AB010BD000000B5A9B0EA
:101950006846FFF7A7FFDDF882000449884202D1FC
:10196000012029B000BD0020FBE700003412CDAB00
:1019700010B50446206807490840B0F1005F08D15F
:101980006068054908602068FEF70FFC024800689F
:10199000804710BD0000FE2F1C00002000B5A9B03C
:1019A0006846FFF77FFF0548CDF882006846FFF7DD
:1019B00083FF0A20FFF70AFF29B000BD3412CDAB28
:1019C00070B504460D46164603496018324629464E
:1019D00000F010F870BD000000000C0870B504465F
:1019E0000D46164604F100603246294600F002F822
:1019F00070BD00002DE9F05F07468846914600253E
:101A0000BB464446AA461DE0E0780606A07846EAB2
:101A10000046607846EA002620780643241D2846C2
:101A2000691C8DB20C4941F82060B5F5007F07D1E3
:101A300000254FF400725846FFF77CFB0BF5006B56
:101A40000AF1040ACA45DFD325B12A46024958469D
:101A5000FFF770FBBDE8F09F6C560020FFF7FCF924
:101A6000FFF76EF9FFF732FF04E03220FFF7CEFEFA
:101A7000FEF780FFF9E7000010B588B004460121A9
:101A80000420FFF75FFA01212020FFF76BFA0822FC
:101A900006212548FFF723F9082207212248FFF7EE
:101AA0001EF9C020069002208DF81C008DF81D0044
:101AB00000208DF81E0001208DF81F0006A91A488D
:101AC000FFF7C5F802940020ADF80C00ADF80E0049
:101AD000ADF81000ADF814000C20ADF8120002A90A
:101AE0001248FFF7D5FD01211048FFF792FD402174
:101AF0000E48FFF785FD012240F225510B48FFF704
:101B0000A1FD47208DF8040002208DF80500032078
:101B10008DF8060001208DF8070001A8FFF7CAF92B
:101B2000FFF73EFC08B010BD000802400014014061
:101B3000000A08003230323330393133303834342F
:101B400035317A68616F796F6E67000000000000C0
:101B50000000426F6F7400000000000000000000F1
:101B60000000000000000000000000000000000075
:101B700000004174426F6F742E6E6577205570645B
:101B800061746553656E642E63616E207265616475
:101B9000207665722066726F6D20617070000000A3
:101BA0000000000000000000000000000000000035
:101BB00000000000D41B000800000020BC01000051
:101BC00050020008501C0008BC010020D474000022
:101BD0008017000801242D010203040436060708BB
:101BE000090113AD021208190932022AD50C31324B
:101BF000034BC1030C2A04244A042432051AE50CC1
:101C00001A010C32061B85050C3132071AC90C2942
:101C10002429355AF90C320B4BC5060C320C4B6992
:101C2000070C2A0D48590C32114B65086C2A15789F
:101C3000190C295432C14B1F091801C81808323039
:101C400032322D3031033D2030303A0321627700AB
:040000050800018965
:00000001FF
